:020000040009F1
:280000000108006999994204204EB1FD0400FFFFFFFF4006000000A0027020020A00280009000000000000001D
:FB002800411A0042726F6164636F6D20426C7565746F6F74682044657669636500980100035C0100017206000300000800017A020000089304002000000068040012000C006A3600030112000000B0000000A0000000431008045310020180000000900000006310040273100402C1000000D000000020000000300000007C04000100000209080068000F0003000000690200BB005D0C000A64E6B000008898425A33435F09003C280100040004F70C0A6E0088010800C600F3025D0066033000C900E10268005C033600C300E2026A0053033C00C200E1026C004E034100C500D60272004A034300C300CE02790042034800C500C00283003A034E00C8002B
:FB012300BF0282003B034E00C900BC0284003703520008080707070707070606060605050505C0E40094FC0E00FFFF00005E02000030FC0E00FFFF0F006304000000FD0E00FFFF0F006602000088FC0E00FFFF0000000200002CFC0E00FFFF00004904000070FC0E00FFFF00000B09000074FC0E00FFFF00002E010000D8FF0E00FFFF000062190000D0FC0E00FFFF000020C90000C8FC0E00FFFF000038850000DCFC0E00FFFF00001CC80000CCFD0E00FFFF0000048000005CFC0E00FFFF00000200000020FC0E00FFFF000019210000E0FC0E000080000000000000C0FC0E00FFFF000022000000C82D08000000FF0000003200189608000000FF00000031
:FB021E00060068000F00FFFF000003080000C314001265141B783F0424306070047180764A3108290ACF090010E0206EF0B009F0601A2400FF0008080312FF10FB0EF70CF30AEF08EB06E7040312FF10FB0EF70CF30AEF08EB06E7040301000182D600FF0602020A233C5A6E7D80008000800080008000800080008000800080008000800014FF1B840AFF200000000000000000000000000014FF1B820AFF430000000000000000000000000014FF1B000AFF660000000000000000000000000014FF1B050AFF660000000000000000000000000014FF1B0B0AFF430000000000000000000000000014FF1B0D0AFF20000000000000000000000000004100F2
:FB0319000000007B0000000041000000007B0000000041000000007B0000000041000000007B0000000041000000007B0000000041000000007B000000008612000413004008000040130001000180FF000112C15E0044041422A244041422A23B04B104B204B304B404B504B604B704B804B904BA04BB04BC04BD04BE04BF04C004C104C204C304C404C504C604C704C804C904CA04CB04CC04CD04CE04CF04D004D104D204D304D404D504D604D704D8280C000B0400665409000823000054A901007AF082FE14005C560900D37A002B04D0937A002B01D085F777F985F780F9082F0001ACB100008AF060FA2000705609005810011C2A1CAB32137800202D
:FB041400994200D2581A05B4201C75F79DFE05BC75F79FFD082F0002C8B300008AF062F9200090560900037D042B09D0052B07D0082B05D0092B03D00A2B01D075F792FE75F7AEFE0000081B0003FC27030063F038F80C00705809000FB400F003F80FBC9CF7D0FF08170004D08E01007CF0D4FD08007C5A090000F006F8FFBD00000B0400845A0900080F0005FC81020000B5000000000000000008170006008202006DF0B2FF08006861090000F002F800BD00000B0400C8610900080F0007143C020002238648000000000000081D00082C6C00008FF0B8FC0E00A06509006EF7C1F8301C207D092870F741FB083100099012010085F08DF92200AE6509B3
:FB050F000003B400F01EF8002805D003BC041C0C2C05D27AF768FE03BC00207AF779FE7AF776FE0813000A9850010081F09AFA0400D06509007EF76EFD082B000BB08701007DF010FF1C00D465090007B400F094F8002802D007BC82F7F3F807BC75F7DEF9221C82F7E8F80817000C78DE000088F068FC08004C67090000F002F810BD00000823000D085B010080F050FE1400AC670900386873F746FC2968386800F003F87FF7A8F900000817000E501F030064F066FC08002068090000F002F89BF7B6FB080F000FBCD20000430700B500000000000008170010C0D2000089F040FB080044690900FFF7EEFF00BD0000082B001100D9020069F02EF81C0010
:FB060A00606909000FB4311CFFF7F2FF002801D00FBC71BD0FBC6946033196F7C5FF0000082B001238CE020069F0AAFD1C00906909000FB4391CFFF7F2FF002802D00FBC96F7A1FA0FBC0902627996F748FA082900138CC002006AF09FFC1A00CE6909001FB4301C211CFFF7EAFF1FBC002B01D195F757FB95F766FB000008170014FCB102006BF040FC0800806A0900FFF7B2FFF3BD0000082B0015587102006FF0BEFC1C00D86A0900FFB402993A1CFFF7D3FF002802D0FFBC90F73EFBFFBC90F73DFB0000082F0016887702006FF0F2F92000706B09000FB4281C211CFFF7BDFF002803D00FBC042090F760FE0FBC984B9D4290F7FEFD081D0017C8530124
:FB0705000081F091FD0E00EE6E09000FB4201CFFF7E1FF0FBC7EF76BFA08190018B41B010085F0B2F90A001C6F0900201CFFF7EDFF7AF756FE082D0019E813010085F09DFD1E00266F0900417B002D06D1238E0F2B05D0042901D17AF75DFA7AF75FFA7AF759FA00000817001A9C5C020071F008F90800B06E0900FFF7D0FE70BD0000081B001B784D020071F05EFF0C00386C090011438173FFF7A8FF8EF79CF80817001C844D020071F05EFF0800446C0900FFF7A7FF8EF7A4F80817001DA44D020071F052FF08004C6C0900FFF7E2FF00BD0000080F001EE052020000B500230000000000000815001FE452020071F0C4FE060070700900FFF768FF00BDE1
:FB080000081900201057020071F0B1FC0A00767009002878FFF77AFF8EF76CFB081700213459020071F0A4FB080080700900FFF7ACFF8EF758FC08170022E85B020071F04EFA080088700900FFF7AFFF8EF7E0FD08170023944E020072F04CFB0800307509001370FFF7ADFD00BD081B0024404F020072F0FAFA0C0038750900281C311CFFF7B1FD8DF721FD081B0025B04F020072F0C8FA0C0044750900201C301CFFF7D9FD8DF77AFD081D00269C50020072F058FA0E0050750900F8210851201CFFF72BFE8DF7A1FD08170027DC50020072F03FFA08005E750900FFF734FE8DF7FDFD081700286851020072F0FDF9080066750900FFF770FE8DF740FE084E
:FB08FB00190029F451020072F0BBF90A006E750900FFF7E6FE8DF771FE00000B0400745509000823002ACC8A01007EF094FD1400F875090002487060024B81F767FAC046BD750900238A0100081F002B348B01007EF03AFD1000AC7509000FB4FFF7E3FF0FBC051C81F7E3FA0000082F002C788602006EF0C8FF20000C76090000B56CF736FD044803681B0702D51E230248037000BDC046E407080003020800080F002DF01D030000F00CF8000000000000080F002E3CBF00004B4964200000000000000819002F1C9004004EF006FB0A002C76090001D0B1F724FDB1F7F8FC0829003030B204004CF001FA1A003676090002D1B3F771FC03E0012903D100BD
:FB09F600F005F8B3F707FEB3F7F5FD0000082100312CA504004DF0ACF8120088760900012098550EB400F023F80EBC207BB2F74CFF08250032B0A104004DF073FA16009A7609005023E05C002804D1206B002801D0B2F785FDB2F789FD08290033286A040050F042FE1A00B0760900116806B400F015F806BC002801D0CB7B00E0E378E078AFF7B2F9081D00341469040050F0D9FE0E00CA76090001B400F010F8011C01BCAFF720F908170035F09304004EF08EF90800107709005C408868B1F76EFE0813003678B104004CF0CEFA040018770900B3F731FD08250037585F000091F0E0FB16001C770900002A06D0039A002A01D16EF719FC6EF71DFC6EF707
:FB0AF10022FC082D0038C862000091F033FA1E0032770900002908D0054A237AD15C002901D16EF7C4FD6EF7C5FD6EF7FFFDC0BF0500080F0039248D0000052924D8000000000000080F003A708D000006E00C290000000000000815003B349300008EF08CFA06005078090000F004F8F0BD0815003CA89300008EF055FA06005678090000F048F8FEBD0815003D10AD04004DF04EFC0600B0850900FFF781FEF3BD0815003E84AC04004DF097FC0600B6850900FFF717FFFEBD080F003F047B040014E0001C000000000000081500405CB604004CF0E2FF060024860900FFF775FD30BD08150041E066000091F0A3FF06002A86090000F001F833BD081500C2
:FB0BEC00425C1D030066F0D6FC06000C870900FFF7D2FF30BD0821004338A004004EF06BFB1200128709000323E374272001230355201C6EF777F810BD08170044B49802006EF036FF08002487090000F002F8F0BD0000081500454C7A040050F0B0FE0600B087090000F004F870BD081500464080040050F0B9FB0600B687090000F06DF800BD081700473477000091F0CAF80800CC88090000F002F8F0BD0000081700484482040050F078FC0800388B090000F002F8FFBD000008150049B0CD04004CF083F80600BA8E090000F010FB00BD0813004A94CE04004CF036FB04000495090030BD00000815004B74BC04004DF080FC060078950900FFF7C6FF39
:EF0CE70070BD0815004CD8BD04004DF0D1FB06007E950900FFF7D2FF30BD0817004D4C48010085F0F6F808003C9A0900FFF7FCFD7AF7FBFF0817004E8CCE00008CF0DAFD0800449A0900FFF772FF73F77AFA0815004F4CD103005CF0F0FC0600309B0900FFF795FF30BD081F0050A4D103005CF0C7FC1000369B09000FB4FFF7BCFF0FBC6CF715F8A3F731FB08170051ACD103005CF0CBFC0800469B0900FFF7B9FF08BC1847081B005228B103005EF011FD0C004E9B090030B4FFF7C2FF30BCA1F7ECFA0829005300BA03005EF0ABF81A005A9B0900FFF7CCFF012801D0A1F794FF024C2078A1F74BFFC046586A0800FE00006F
:FB53000030B55F4C5F4B604A13606048036804221343036005205E4A10600F2212041368F0218B43136050231068184310606AF7A9FF051C574B9D4201D3AD0803E05B109D4200D36D0854486843544941185448C0F7A0F9411E4906090E402902D3DF310906090E18209DF749FB68084D494118281CC0F78FF9051FB2209DF74DFB382188436907890E014332209DF737FB90209DF742FBE0218843382129408900014310209DF72BFB40490B6840490B6040490B6840490B6040490B6840490B6040490B6840490B6040490B6840490B6040490B6840490B60E06D3F4908603F490B683F490B603F490B683F490B8000233F490B703F490B703F490B683F0A
:FB53FB00490B6023683E490B6060683E49086020490B685B031AD43C4B3C4803603C4B3D4803603D4B3D4803603D4B3E4803603E4B3E4803603E4B3F4803603F4B3F4803603F4B40480360404B40480360404C414B236502F0A7FA01F047FA3F4B23603F4B3F490B6030BC08BC18473E483E49086000233E490B70FF233D490B7002233D490B6070472CFC0E00C555090054CE0800100B0800400B0800E0AB0000577C000050A06E00A040DD00C0450400D8FC0E00902D0800E0FC0E00942D0800CCFC0E00982D0800C8FC0E009C2D0800DCFC0E00A02D0800D0FC0E00A42D0800842D0800CCFD0E00882D08003CFF0E004CD208004C9E09004D9E0900D4FF1E
:FB54F6000E00849C0900889C09008C9C090050850000A802080007470000AC02080038850000B402080041450000B00208001CC80000B802080020C90000BC0208001E450000909C090049070000949C090069040000989C0900281B0800FD77090023660900020A0100040208000153090090000800720808004E9E09009C9C090070B500200F49104B4B6114E05A099200DB06DB0E01259D408B582B438B504B694200C50064196468012634432725AD032C1B9C520130054CC300E358922BE5D370BDC046D41B0800489E0900B49B090030B5194D01244A7812020B781A43AA4202D100F06BF823E0144B9A4202D102F0B5F81DE0124B9A4202D103F0C932
:6B55F100FF17E0023B9A4202D103F0E9FF11E00D4B9A4207D10D490B7F002B09D00D230370012007E00A4B9A4202D103F0E2FF00E00024201C30BC08BC184714FC0000030C0000C6FC000005040000B8210800C8FC00000B7B1B065B0E3C2B01D10248886000207047C0461B6709006D
:FB56B00030B50C1C664AD36A032000068343D3620723644A13600025E378002B00D08FE0012561480378002B11D1012000F003F95E494B69DB07DB0F5D490B705B494B6901218B4359494B61012357490B706079012807D30AD003280AD30ED005280FD312D015E01C208543182010E051480EE05048054302210D430AE0E020854307E0E0208543202002E0E0208543A0200543A1790320800285438807000D05430120002900D1022000F042F9E378002B47D13E4A5369012293433C4A5361202147209DF744F9BA2146209DF740F9472000219DF73CF9C8209CF7E2FB082147209DF735F964209CF7DBFB282147209DF72EF9C8209CF7D4FBBA2147209D65
:C557AB00F727F964209CF7CDFB217941209DF720F9E379072B05D85B42980600167FF76DF909E0082B02D10823E056F7E7092B03D1607A7EF75CFF031C1906090E43209DF707F924E0412000219DF702F9432000219DF7FEF8462000219DF7FAF8472000219DF7F6F8114A1378002B10D0002000F064F8104A13780E4A506901229043D907C90F08430A4A50610023084A1370E378002B03D009480540222005430848056030BDC046D820080058D208004C9E09009C1B08004D9E090000010000FEFF0000C0FC0E0093
:FB587C00E0B565496548664A664B674D674E684FEEC01838674A10600F23674A537088209DF7BCF8654B664A13600007000F00F04CF890F75FFD012000F017F8614A1378614A506902229043D907890F08435E4A5061A4F7BDF85D4A13689B0301D4ABF74DFE002000F001F8E0BD30B5051C584C04F042F9012D15D1002356490B60012355490B60802355490B60554B1D21C9030B60544D29680A06FBD52368012149040B430EE022234C4A136023680121C9050B432360002132210139FDD123684A490B40236004F020F930BDF0B5474B5A33C45C474D1022281C002104F01DF900220A20604341494118D300EF1834480368181C3F239B0218400B881898
:FB5977004338808B889806030C48881843788088880F239B0103409E110B8903200002034018123303CE88B60033431843B8800B891E06360C304803681806000E3043F88001321206120E2D480368E41A2406240E022AC7D302201E4A13685B0300D5012000F001F8F0BD10B525490B78834214D00870012801D0032801D1002000E001201049C3001B48C25AC0180A6042884A6082888A60C388184C236010BD49960300A09C0900B7960300DD96030059970300ED600900EF9803000C0C08009C0B0800C518000054FD0E00AC0B08009C1B0800100B080060000F0000820E00C0FC0E0004820E000100800008800E00FFFF7DFF88010800389E090060FD6E
:0A5A72000E009C9C09004E9E0900E6
:FB5A8400C148C24908607047C14908780130087000060CD1BF4AC42300209850111C5031FF230B5401300928F8D37F234B727047F0B58EB0B8490791B8490B7801330B70002842D1B648A92189004318B549415CC956002901D0B44AD17600268257002A03D1B2490023CA568255AA4C251CB04F0197012179568B185B2169565035994206DA07217B569A4202DD019B197803E0A15D002901D00139A155032179568B180B216956994207DA07217B569A4203DD7434BB78335505E07434A15D002901D00139A15501364F2EC8D3924C251C50350A22291C0BA8BFF765F90026A35D002B03D1311C0BA800F0FDF901364F2EF5D30026221CC03200920123B38F
:FB5B7F004006935068034029D08B49B300CA180492136819058A0E05929906890E08A800F026FA002708AB0BA9CA5DD85D10409CF7A3F90599091A05910A1C01370A2FF1D304990B681B041B0F5800111C814205D20699CB4300994868184048600136162EC9D307990BA800F0DEF9A872000600D046E1704883689B0711D5281C18308DF74DFE4F21281C183000F0B7F9291C18310BA800F0C8F9A872000600D030E1002606960A22FF21281C0C3003F0B3FF4F21281C0C3000F0A1F90596211C733104910E70211C723103910E70002102915B4909688F5D5A480268905DC31901B40698984201BC00D20593002E06D14B7809785918537812789A1815E0F9
:FB5C7A004E2E07D14C318B78497859184C3293785278F3E771184B1E49781B78CB18F918B3185F1E5A783B78D318C218434F01975318787983420DD938790B1C4343FF21091A51438B4205D2012102910398037801330370311C281C183000F037F9002809D0231C7433F35C002B04D0049803780133037002E00298002804D0311C281C0C3000F03DF901364F2EA1D3B87905990023814200D901230099CB7000260120B040009A5168084011D02449B300C9580A05920E8906890E08A800F05BF908A90BA800F045F9A872000600D09BE00136162EE4D3002602960123B3400098416819404AD11649B300CF18049739680B059A0E8906890E08A800F03C4A
:FB5D7500F939680905880E0390002708AB79190A7BD85D10401BE0B55A0900201B08004F9E0900B89C0900DC200800509E09003433080013030000F89C0900139D0900D89B0900E49B0900380408003C0408009CF798F80399091A039101370A2FD5D3049803681B041B0F081C5900884207D30121029106980399884201D2069105960136162EABD30298002828D0B049059EB300CF1839680B059A0E8906890E08A800F0EBF80123B340009E70681843706008A90BA800F0CFF8A8720123F3703B689906890E0E1C03E001980378A35501363B681B059B0E5A189642F5D313E0291C0C310BA800F0A5F8A8720026311C281C0C3000F076F8002802D0019866
:FB5E70000378A35501364F2EF2D3AB7A002B33D0002708AB7819007E079AD15D0840D85501370A2FF5D30693181C83F7A0FB142801D807980690AF7A1CE00026A15D002903D00139A155090611D1311C0BA800F04AF800280BD0311C069800F03CF8002805D0311C0BA800F047F8013F04D001364F2EE3D3002FE0D10A220BA9281CBEF79BFF00260324311C0BA800F024F8002800D00124704D221C311C281C00F03EF801364F2EEED3311C281C002200F036F883F784FA69488368DB0701D500F091F80098C378002B01D082F742FB01200EB0F0BC08BC1847CB084907490FC05C0841C007C00F7047CB084907490FC05C0841C307D81701307047CA084B8E
:FB5F6B00075B0F01219940835C0B4383547047CA084B075B0F01219940835C8B438354704730B50B07DC0E090989000323A34045589D43A2402A43425030BD10B50022835C8C5C2340835401320A2AF8D383F711FB0022142801D214231A1A101C10BD10B50022835C8C5CA343835401320A2AF8D383F7FFFA0022142801D214231A1A101C10BD70B5CC085318DA084E07760F5D076D0F002102E0002343540131A142FAD9311C05E001238B40065D1E43065501310829F7D3611C02E0FF23435401319142FAD9291C05E001238B40845C9C43845401310829F7D3511C02E00023435401310A29FAD370BD70B5FF25CC261D489BF780FB041C42D025700E23BA
:FB6066006370A6700123E37019494F2301205854C822201DBEF7D5FE14221149201CCC30BEF7CFFE50221249201CE030BEF7C9FE502210480168201CFF303130BEF7C1FE50220D480168201CFF308130BEF7B9FE064A211C0A4890F720FA12E0C046E49B09000C470800D89B0900D0010000B89C090034330800380408003C040800C050080070BD000070B50024ED209CF791FC4106490E6D209CF77EFCEB209CF789FCC506ED0E63071B0E1D43ED209CF781FCFC21014018202040C00801436D209CF76AFC291C6B209CF766FC002C04D10B4E35682D68C5F7B4FD62200021A3F75DFA002802D00134192CD7D9044E3568ED68C5F7A6FD201C70BC08BC18B4
:0761610047C046C00B080017
:FB61700010B5C3699B0121D5C17B03291ED9038E0F2B0BD1042909D100214B000D4A448ED25A944212D001310429F6D3006887F785FF0368002B00D00123002B08D0037C122B05D144300078002801D0002000E0012010BD3C9C0900A848A94988657047F0B583B0A74EA84CA84DA94F3F6801963E60BC60FD60A74C02947C60A64EB407A40F01D135680CE0361BE4003568E540009520252C1B7568A54001B40198054301BCEC0F9D4D2C70002F07D0012C01D1019C00E0029CA446C5F744FD03B0F0BC08BC18470023964803700123954803700023954803609548036095480360282394480360072394480370302393480360704700B5FFF7E6FF8DF7F1C9
:FB626B00FC864A9007800F01D1116808E0121AC0001368C3402021081A516881401943090105D588480368022003438648036008BC1847000000B5FFF7C7FF8DF710FD774A9007800F01D1116808E0121AC0001368C3402021081A516881401943090104D578490B68022083430B6008BC18470000F0B581B0744E0024271C0090684A1378002B7BD075682D0C2D044B006F4AD25A002A01D1141C6FE06D4B1B68002B07D0602A01D1E0221BE0702A05D1D02217E0042901D101242404302A05D16C23195C002901D0634A0BE0502A09D100990B6FDB0503D501235B041C4301E05E4B1C4014435C4B9A4202D013095C49CF5C302A0AD16C23195C002906D15C
:FB636600011C28310B7D897A5F183F063F0E3B031C43C37B002B02D00123DB031D43C37C032B04D1818CCB06190F0B021D43402A25D13E490B78002B05D000F0E2F803071B0A1C431BE00123DB041C43009A907B9BF77FFB4008374A1060354A11689BF714FB354A1060354A1368984204D2009800F0A4F8002802D001232C4803703460756001B0F0BC08BC1847F0B582B001900F1C2E4E00210091051C132F77D134682348017800291AD1A87B9BF752FB4008214A10601F4A11689BF7E7FA1F4A10601F4A1368984204D2281C00F077F800284ED0012316480370234B1C4048E06B6E1B0645D4012943D1281C00F067F800283ED1A87B9BF72DFB41080DF1
:FB6461004A116000230B4A137031E0D1610900201A080063620900DD620900F1630900C4050800A16209004405080050CD0800519E0900529E0900809D0900849D0900889D09008C9D0900539E0900909D090070010F0070820E0058050800C4C9080080010000FFFFFDFFA4050800FFFFF7FF0123DB041C432B480378002B03D001988CF7FDFF0090284B1C43009803071B0A1C433460042F05D13368012109040B43012107E021480378002B06D0336820490B40002133601D48017002B0F0BC08BC184770B5041C6434207F430119495D1877F747FC061C2D68002D13D0EB68002B10D4207F93F743FAEB68190109099BF74FFA90363188104B1A68891AB0
:44655C00884201D3012000E0002070BD10B5041CFFF7D9FF002802D00949087802E0201C8CF7AFFF10BDC046529E0900FFFF0FFF519E0900FFFFFEFF542A0800909D0900539E0900C0
:FB65F00070B50E1C0124051C77F7E3FB31784B10072B0CD14B4A11884B0708D50123AB40494A118C194002D091F799FB0024201C70BDF0B583B04548037E002B65D1424CE369FE20034060D04149C87C431C1806000E77F7BEFB051C83F70DF800280CD10126301C77F7B5FB051C83F704F8002803D10136082EF4D347E0002D45D06946281C82F70BFF002804D03249887882F742F83AE00126301C77F79BFB051C82F7EAFF00282ED0286875F7E1F9002829D1286801238340218C194023D16EF79FF90A226946843003F075FA00281AD0029B0120C00703430293EB691B06DB0E072B02D2EB6C002B0DD4281C82F7C1FB071C3A1C6946281C75F75EF93A68
:6166EB001C6946281C82F7C3F90136082EC5D303B0F0BC08BC1847011CCB6900201B06DB0E072B03D2CB6C002B00D50120704700B50A4A012301688B4011881943118075F7CBF908BC18470000DCC908000C470800F42D0800343608004C0408002C47080042
:5867540010B50124201C77F732FB00280FD0C3695B070CD0C06CC000830F032B07D103F0FFF9041C0A490B690A48034309E00134072CE7D903F0F4F9041C05490B69054883430B616FF718FA201C03F0F1F910BDD820080000000020FD
:6067C000F0B581B0814227D000256B00134A9C1801278740FE436388334063801A1C63893340638101238B401E1C134002D03A4362806288F34300931A4062806289164002D03A4362816289009B1A40628101352D062D0E032DD8D301B0F0BD0CCA0800D1
:FB68280070B5051C114801688023194002D0104E002409E00C1C02E09BF7D8FB0134AC42FAD311E0AD1B0134731C9D42FAD206E0B6F776FC301C9DF7B0F8B6F776FC013CF6D2281C9DF7A9F870BDC04608A00F00D3300000F0B5071C00263D1C1D4803689B0724D52C1C50340123E3731A4BA87B185CA37C022B0DD118480378012B07D8174A13689B0603D50670022071F7BDFC266001E0032803D20D232B745423AB74637B002B03D00F4803680F480360AE81381C8BF766FFF0BC08BC184710B50B4C2C220B490B48BEF79BFA0A4884610A4B186010BD2C8B0E0051C5080045220800BCC90800B804080028FC0E007D680900A0CE0500949D0900C40408BB
:216923000000B5431E044A1360044A13685B0301D4FFF753F800BDC046E08A0E00100B0800E1
:14694C00F82213585B0703D50C230B70012000E000207047F6
:14697C00F82213585B0703D50C230B70012000E000207047C6
:2269AC00F82213581B070BD5C3691B0408D44B7A012B05D1F8221358FF2101310B431350704715
:9869E800F0B582B0051C0E1C00230193301C77F7E4F9041CE3695B0409D56B4601AA211C4C31283097F735FF002800D12FE0032094F783FB071C2AD0301C77F763FBF8725C231E5B211C2831781D0622BEF7F8F9002D04D1311C201C2830A2F758F8BD70FE70300A387198221359DB00DB0F3B73381C94F7E3FAB978002905D1054A536F0120000483435367201C00F092FC02B0F0BDC04658210800E5
:506A880070B5041C0D1C161CF82003595B0719D5E3691B0416D40C4803689B0712D5201C283000F0F0FC3104090C281C90F7F4FB0821201C7EF7A4FA8EF702FB0120034A107000E0002070BDEC1B0800549E09002A
:7C6AF40030B5041C0D1C30D0F82108590007830F012B2AD1E3691B0427D42B7B1B065B0E23D01349086880071FD5201C283000F0B4FCF822135902229343F8221351281C9AF7F4FD0821201C7EF764FA8EF7C2FA0123084A1370084A1168201C8EF7B1FA201C00F017FC012000E0002030BDC046EC1B0800549E09005052080046
:A86B900025494160704710B588B04468E269130408D4201C8EF74FFA204A1168201C8EF782FA2DE053055B0F01A88370E3699B045B0FC370E37B07A80370636B0293A36B0393E36B0493236C0593201C5030038806A90B80C378CB7083788B70A37E07A84370E37E83706846831D19220C48002194F7CCFC201C8EF71EFA00230948037008B010BD00B54068F822135840210B4313508EF7E5FA00BD0172090050520800B5FC00008CCD080059
:FB6C540070B582B0002301938D490868042826D18C49086877F7ABF8041C5C238A4908881853E369F820834310200343E361F8210B5904210B43F8210B518EF710FF814908687BF7B9FDFF237E490B60F8210B59402003430B51201C8EF7A0FAEEE0022841D1784A106877F782F87849041C8EF761F9F8210859030704D5031C02218B43002002E0022303430120F8210B5101218B4308400343F8252B518EF7E0FE02F03FFF012321688B40694A11681943116002F03EFF20686DF7CAFDE369AB4310200343E361206801216DF733FFFF235D4D2B60201C91F725F8201C8EF70BF8201C8EF791FAAAE080280CD1584876F714FD002800D1A2E0C369F8218B51
:FB6D4F004310210B43C3619BE0202800D198E0102857D15149086877F72CF8051C4F4E301C76F7FCFC002811D0041CF822135901221343F8221351EB69E06907210B4088431843E061286876F779FF0CE02C1C311C201C28300622BEF73FF8F820035902208343F8200351311C201C8EF7E5F8002805D0F820035901200343F8200351201C8EF743FA02F0CEFE012321688B40314A11681943116002F0CDFE20686DF759FDE369F820834310200343E361206801216DF7C1FE201C90F7B6FFFF23264803603EE0FF230133984236D1244876F7A6FC041C35D077F713FAE369012000068343F820834310200343E361E36C5B005B08E364EC210B590006834358
:666E4A000B51201C00217BF726FA201C00217BF77DFA6B4601AA211C4C31201C283097F707FD002806D0019B002B03D0201C7AF767FE03E0211C002077F744FEC0E7402801D18EF7A0FE02B070BDA45208002406080054520800BFC60800ACC9080028060800B052080070
:366EB80010B5041CF82003595B070CD508225C23195B101C94F76AFAF820035904208343F820035106E09A231A5D5C342188002094F75CFA10BDE5
:206EFC0010B5041CF82003591B0708D4201C7AF71EFEE369F820834320200343E36110BD95
:FB6F440034480023344A136034494167344A13600360344A13605360334B344A1360344B344A13604923344A1360704730B5334C3349022823D004282DD132480368180A031F0218D01C2060636008606068486000232D4D2B602D4803682D4A1360436853602C484178CB0101781943807883030B4311070B43284A1020011C08E049204860264A1368802003431F4A1220282113606EF7A6FE30BD00B5002320490B708EF77CF900BD00B51E490868FF2804D076F74AFEFF231B490B6001231A48036017480378012B04D18EF759FD002314490B7000BD18800E00F8800E00447E000098830E0040820E00FFF2011A94830E0040C07DC0D4890E00148B0EB7
:31703F0000449C0900108B0E0034060800A4860E009C52080018820E003C060800009A0E00AC520800549E090028060800A45208004F
:FB70900000B50021B34801700C22B34802F07AFD00BD30B5041C24234B43B048C518211C2831281D0622BDF7B7FEE3695B055B0FAB72E3699B045B0FEB72E37BAB77636BEB60A36B2B61E36B6B61236CAB61201C503003886B80C3786B7783782B77A37EEB772023E17E595583892B8030BD70B50D1C022D52D2041C77F751F824236B439648C518AB7AE0690722120290435A07520D1043E061EB7A0722D20290435A07920C1043E061AB7FE373EB6863632B69A3630822291C1431201C3C30BDF76CFE201C50306B8803806B7FC3702B7F8370EB7FA3762023595DE176E3690F21C9050B43E3610F232386F4347D490A685206520F226086892C88A64205F9
:FB718B00D0794A0121B14013688B431360764A01210B1CA34015681D4315608481081C00E0002070BD00B5F822135840218B431350C3691B0402D4002100F030F900BD70B5061C351CFC352C68002C03D0201CB6F745F80AE014209AF787FA041C09D02C60321C62490023B6F71AF81421201CB6F721F870BD00B558490B78012B04D18DF7F1FF002354490B7008BC1847000010B5041CE3691B040BD42068431E0B2B07D2F82003595B0703D55C23185B76F7BBFC13225C342188002094F7AEF810BD70B5041C0D1C161CFF2001302058002801D0B6F704F8F8200359DB0745D5002D43D0002E5BD0F82003599B0757D5201C6DF749FCE369F82083433820DA
:FB7286000343E361F820035904208343F8200351201C90F7BDFD206800216DF771FC5C23195B00231A1C181C94F7D3F9201C28308DF7EFFDE3691B0407D48DF701FE00F0C9F8012801D100F018F900232A490B70A36B1B072FD5E3691B042CD427494B681B0528D5201C012100F09BF823E01E4803689B0715D5F8210B59082003430B518020E3691B0400D440001C4908600120000777F786FB002D0DD1201CFFF77AFF09E0E3691B0403D5201C8DF75EFF02E001230A48037070BD10B5041CE3691B040BD48DF7BDFD00F085F8012801D100F0D4F80821201C7DF754FE10BDC0467C9C0900559E090054520800EC1B080054210800994D02008CCD08009C34
:FB7381001B0800A452080000B5FF2101314058002801D0B5F768FF00BD70B5041C0E1CB625F82003591B0600D5D025F8210B59802083430B511807830F34D0002356490B70F8210B590C2083430B51201CFFF7DBFFE3691B040CD5002E24D0311CAB059B0D3F208002184300231A1C94F7D6F819E0F8200359DB0509D5F8221359FF20013083431351201C002194F70FF98DF75AFD201C283000F05AF800F01EF8012801D100F06DF870BD10B5041C012906D1012181F780F9201C81F7FEFC0CE0E4210B590120800483430B513448012221688A4003689343036010BD10B582B006222F496846BDF7E0FC00246946062363432C481818062202F095FB002874
:B4747C0001D0012003E00134022CF0D3002002B010BDF0B582B0071C062224496846BDF7C5FC0024204E0622151C65436946A81902F07AFB002806D1391CA8190622BDF7B5FC012003E00134022CEBD3002002B0F0BDF0B5071C0024134E0622151C6543391CA81902F060FB002806D1A8190622002102F051FB012003E00134022CEBD30020F0BD00B501230448037008480368022B01D18EF7D7FA00BDC0468CCD080028470800C49B0900559E0900CC9B090050520800B5
:3475780010B5041CE069C30B2121194020290DD10306DB0E062B09D8054803689B0705D4201C81F74DFC201C7AF73EFB10BDC046EC1B080025
:3C75BC0010B5041C74F763FA0B490B689B070FD5E069C30B21211940202909D10306DB0E062B05D8201C81F729FC201C7AF71AFB10BC08BC1847C046EC1B080025
:3876500010B50A4C2168012292030A432260084C2368DB0608D54A0406D4036D186BC00602D501230348C37710BDC046808B0E0008800E002422080009
:3876D8000B490B680020D87370470A490B7C0020002B00D1012070470120054A1368D97B002904D1034A117C002900D1081C7047B0A20800986308007A
:FB77500030B5041C1E480368002B04D0002303602823002018551B4D00216962A96279F7DDF819480368002B03D176F7E6FA002803D1012093F7FCFB04E077F772FA2834042020700023114803701148037801210B43037099F771FC281C8A300622002102F0F0F90B4803680B4C23600B4C23680B4C23600B4C23680B4C236030BDC0465CCE0800D82008005CD20800ADC50800140B0800849C0900D4FF0E00889C09002CFC0E008C9C090030FC0E000C49012807D10C4A13680C4A13600C4A13680C4A08E0002809D10B4A1368074A13600A4A13680A4A0B601068486000207047C0462CFC0E00909C0900D4FF0E00949C0900989C0900849C0900889C0902
:05784B00008C9C090007
:FB785C00F0B583B0051C4A4F2E1C1836009601A9A87B9AF709F931684A000198824201D3141A02E0831A434AD41AEB7C032B23D17B1C9C4219D940089AF7ACF8B489011C201CBDF7F9FE0130012818D0031C634300990868C0183840086042000198824201D2801A334A141A0AE0022C08D8324803699D4204D002E07B1C9C4200D900246108281C71F7C0FC201C03B0F0BDF0B583B0061C294F351C183501A9B07B9AF7C3F8A87B019C830702D50123DB065C406889002807D04000844201D3241A02E07B1C001B1C1AA9890091600875F793FB009A131A5800E307DB0FC41AEB7B002B0AD0042C18D9A989019823181F4078089AF750F8002413E011490BD5
:FB79570068702003401809B37B834202D1042C05D201E0082C02D2A8894300E418019823181F40780828606108301C71F76FFC201C03B0F0BDFFFFFF070000001004220800FFFFFF0F24860E00014B0248036070474C9C09009414080070B5041C00216FF769FD061C03D50123B948437147E0E37B012B0FD1251C7835687A00280FD1A07B9AF76EF84008236DB83319689AF70BF8002806DC251C7835687A002805D0002E03DD201CB3F72DFE29E0E37B012B03D1002801D101236B72A87880210143A54A1160082105206EF782F9A14A5379002B15D1B1F76FFA201CB3F706FFB1F789FE0023AB74FF200C30231800201870201CB3F71BFF201C00F0A3FF79
:FB7A520001F045F870BDF0B587B0061C0125341C934902910B78002B17D0E37B002B68D1271C81373B78002B63D105A9B07B9AF700F805988007800F032802D1069B6E2B01D2002855D13D7053E0854B1B680193854B1F689BF746FD0090201C00F0E7FC009BDB070DD47E4803680198984203D17D4803689F4204D09BF734FD0090CD231D550098C30706D57848457430688769301CC4F7DDF8201C00F0C9FC236DBE331878C000724908180379002B21D0211CA4314F6800230E68039604933206120E03B403980590C11706918B4200D1824203BC07D1009A530704D4654BF218654B5F4184C100230371FF200B30231800201870B1F743FE236DBE33182E
:FB7B4D0078C0005B490B580E18002B0CD5E37B012B09D1FF200830205C002804D1A07B99F7A4FF4008306002980378002B08D0271C81373B78002B03D1E37B002B00D13D7007B0F0BC08BC1847F0B581B00027041C251C8035AF81EF76FF230533E618F3790133F371E37B012B13D1F378002B12D1434803689B070ED5A07B99F776FF81084900A069814206D099F70BFF4000686001E000F007FD39480068009083071DD538490B685B0610D5A07B99F75EFF400828846B78012B08D102236B70236D588900016884201CB3F754FCF379012B05D17CF73AFF011C201CAFF797FF00980621014006292BD126490B685B0604D4A07B99F73BFF40082884236DAA
:FB7C4800BE33187887F7CBF9201CB1F7A2F96B78012B08D102236B70236D588900016884201CB3F729FCE37B0099201C002B02D1B3F74EFC01E000F093F9201CB0F73CFFAF722CE0B771830722D5A87A0F490B7898421DD2E37B002B1AD00130A8721EE0082D0800A4860E004322080088830E0090830E0068D20800C09D09000100000000000000BC8B0E005C1408008CD208002B7E002B00D02F76201CB3F7BAFC01B0F0BC08BC184700B50121027D062A02D0072A00D00021002902D000F0B0F809E0037D032B02D100F0DCF803E0042B01D100F0F2FB08BC1847000010B5041C00290FD1B1498B79002B07D0B0490B69834203D146310120087036E02000
:FB7D43001CFFF734FE32E0012905D1201CFFF77EFC00F0C4FE2AE0022923D1E37B012B05D1236B002B02D046231B5BA38100F0B6FEA049CB7F002B10D000239F4803609F4803689F48036000239E4803609E4803609E4803689A48036008E0201C00F02DFA04E0042902D1201C00F068FB10BC08BC184730B5041CE37B002B1CD1211C80314B78002B4AD101234B70A07B99F772FE4008236DB833196899F708FE011C3DD0206D82F770FF236DB0331888608418340123237232E000F0FAFB8548417C01394174417CFF220B32A31800221A70012904D8804D2B68804A13402B6000291AD0211C8031CB7E002B02D1898BCA0612D5007C010712D473490B681A
:FB7E3E00784803400B606D490B68764803400B6076490B68764803400B6002E0201CB3F7FDFB30BC08BC184770B50125041C80304378002B07D10323E37420231D55837E002B00D0C572231CFF3359595E19A06999F7AFFD216DB2310A88011C101CBDF7FAFB011C201C00F076F9A3693360201CB1F76BFC236DBE331878C0005D4908180023F37103715B48057070BD70B582B0051C2C1C8034E37A002B08D02B6DBE3319780820AFF7A8FD0023A376E3726378032B26D0A87B99F7E0FD4108208C0B1A1E04360C618C8E421BD36078012806D1A88CBDF7E4FB062803D13E2002E0042803D008202B6DAF33187003236370281C6EF769FD2B6DBE3319780573
:CF7F390020AFF77CFD31E06068002808D00090002301936946A87B99F7F9FE002363606378032B11D0FF200930285A864209D8A87B87F70BF8002804D1281C00F022FB002802D02E49C8780CE06378002B07D12C4BA87B185C032802D22949887801E027494878A874281CB3F797FB02B070BD70B5051C0E1C2C1C8034A37F002B4ED0B1F7F9F8154A537C012B09D9E37E002B02D1A08BC10603D5311C281CB1F7BEF8CD23585D00283AD0FF230533E8188379002B34D028E0C04644220800C82C08002422080064830E00980208005C000F000E
:FB800800808B0E0014800E009C02080068D208001C800E00FFBFFFFFFFFDFFFFFFFBFFFE608B0E00FFFFF7FFC09D0900619E09009014080051C50800C378002B07D12B6DBE331878C000BD49081801230371BC490B681B0708D56378022B05D1A0898304980E01D10123237670BDF0B5051C2C6D261CB036208B430070881818A969431858014009B0602F1C803700237B700223EB74A861F18899F7A7FCFF2101316850B38833806B84F3887380AB84EB7B012B04D1E07D4300A34858432863E08B03017B84281CB3F7F8F900233B76E37DE370238BA380608BE388834207D16389E18B8B4203D12389A18B8B4208D0E080E38B6381A38B2381236B04210B31
:FB810300432363307B99F7D6FC40083884F0BD30B5041C256D8D4803689C4201D1B1F755FB201C00F0ABF9211C8031088900280FD001380881088904234B70002808D1201C6EF75EFCBE3529780520AFF772FC1EE0487800280CD1B0356888AA68831858014009A86000234B700223E374A0610BE0022809D18B7E002B06D0CB89088A834202D1201CFFF773FF201C6EF7E1FD30BD70B50E1C041C7834E38A9B19E382051CB3F70DFA286D0069C004C00E7043E17809182520BDF788FAE070E1781F2905D90B1C203B01209840237A02E001238B406068184004D16078BDF776FA5435415D584A13689B0607D4E17202200A2900D8012040184000A07070BDCC
:FB81FE00F0B581B0071C3C1CCC34626890680090514E337CFB2003403374391C9C3108883F231B0203401D12737C012B0BD9D368AB4203DCA368DA68002A07DD102318430880088802E0444B184008802178CA07D20F0099B0F766FE737C4049012B25D90B680120800303430B606368D868A8420EDCA368D86800280ADD381C01220021B0F7FDFE2178CA07D20FA16889680AE0291C381C0022B0F7F2FE2178CA07D20F616889686918B0F75BFE03E00B682C4803400B6001B0F0BDF0B581B00090051CB035A97B284B4B4328495C18264A201C002101F060FC1923237400206074234BA17B595C032902D22248817801E020484178A1742B7BA3736B7BE357
:FB82F900732B8863846B88A384A968271C783700227A720223E374A16100982065FA70BB70FA720123BB84261C9C361349CB7CF370FF21073163181148017A1970A97B4D23995561239955331C1BE0C09D0900A82D0800710200000422080068D20800EFFF00001C800E00FFBFFFFF2801000000A4080051C508009014080008960800C82D08003C337363331C5033B363A18C06224A43F280201CB3F796F80099CA68097C201CB3F7A5F8744BFB82AB687366201C0121FFF7F2FE6B7B012B02D1009882F7DEFBFF210D31631800225A70236DBE331978C9006A4A0123DB078B50694A1168201C6EF7A5FA86F72FFE01B0F0BDF0B583B00291FF2329334343F4
:FB83F4006248C618356D01F0BBFB371C90372C1CB034029B8E22925B9A1A1204120C638853433A6FD21851014909019101F0B0FBF37B012B0ED16A8B53000093288B4000019A101841014909181CBDF745F9A080009BE380281C82F795FBF37B002B0ED1E68870086883A188019899F7C7FAE288011C101CBDF730F9301A40082883029B581E38800123BB7203B0F0BDB0B584B03F4C011CCD310B78002B35D000230B7022680192910618D5216A676A0A06394B0B401B021343384A0A40120A1A43090E0A435100490800220D02029703923D430A0E031CA433291C06C3019A510613D5A16AE76A0A062B4B0B401B0213432A4A0A40120A1A43090E0A435110
:C184EF000049080A0E09023943AC3006C004B0B0BD30B5041C256DE37B012B19D12048214A537A5B0029690904490F4900415AC05A08181D4A1378C11A201C6FF73BFBE87843001A4858431A4A11780B18236302E0A07B99F73AFCBE35012128788140154803680B4303601448E37B012B00D1134803680B430360A07B99F7A6FA4008A034208030BDFFFF0000C09D09009414080000A4080064830E0000FF00000000FF0074E50500C82D0800C8020800710200007414080084D2080080D2080088D2080052
:6885BC0030B5041C236DBE331878C00014490B580D18002B0DD4A07B99F770FA4008296899F708FAFF210931615A884201D9012000E0002030BDFF210831431801211970084A13788374036DBE331878C00004490123DB0743500818002303717047C046C09D090090140800F9
:DC86300030B582B0051CAC686946201C99F702FB00998B079B0FFF2239325A430198801801908B089B0000930E490B88984203D30D490B1AE4180191211C0C48BDF712F80130E8830A4A1368E4180A4A136CDB0601D409480460503CEC82084B08490B6002B030BD789C0900E20400007102000014040800C82C0800108B0E00FFFFFF00F4800E00F0B50E1C114D124C28603368DB0701D599F793F90020606627680E483840206099F78EFC99F78CFC3068E8607068A8600220606699F784FC99F782FC99F780FC27600020E860A860F0BDC04600820E001C800E00FFFFFFFD09
:84872C00F0B51E4C2378002B34D0051C6078431E9B00D91D0906090E132092F7E0FC061C25D0A11CF01C6278B2700FE04B781B020F783B4303701B0A4370CB781B028F783B4383701B0AC37004310430013AEDD27422201C002101F007FA002308480370281C01F0F9F9301C92F746FC04E004490E70281C01F0F0F9F0BDC046B85A0800C2CD08007F
:FB87BC0070B506794588281CADF714FF041C701E092860D801A1095C8F44C0460A301EBA6EBA7692B4583648037C002B05D13C210F20AEF7D1FF012005E0002C4BD0281CAFF7E0FF0220AFF710FF44E0281CAFF7D9FF0120AFF7AFFF2A490B680020187029490B78022B36D101230B70281CB3F79BFF30E0281CAFF7E1FF0020AFF79BFF20490B680020187025E0281CAFF7DBFF21E0002C1FD0236B082083432363211C2031201C0C300522BCF7E0FA13E0002C11D0236B0220834323635B070BD5201C0021AEF7C3FF236B04229343236302E0281CB4F7BEFA70BD00B5012802D1AFF749FF0CE00020AFF766FF084800231A1C191C92F775FE0F200221AE35
:1588B700F76DFF00BD98630800BCA2080094D208000E20000087
:FB88D400F0B581B0071C284C261C453600233370264803681B071B0F012B02D12449887B09E003681B0703D122490868088802E00023238736E020490B78C01A20871F490D6820E0281FEB7A012B1BD10168896A0091002101B40198844601BCC3F7C0F900280FD020300379002B0BD0C078032801D0022803D1238F608F834202D00123337003E02D680D488542DBD13378002B08D03D68208F291C41430948BCF790FE281A386001B0F0BD0422080010000F00182108002C0B0800C80208000803080040420F00F0B586B0051C102340490B602F1CCC373878002870D03E4E3E4B3F481861EB7B012B13D13D4CFF200B30285C002808D03B4C9C23585B00B1
:FB89CF000700D53A4C0123DB071C4333688020034333600DE0364C9C23585B3F21090201400A1200D0043212028007800F1043F061281CB0F7F8FD3878C30701D52D4B1C43830729D52C4B1C432C4A107C010706D52B4B1C4333680120C00403433360281CAC3006C804A806C004990806000E254AD0620A0A0598000602431106FF200002104000020143FF2000041040000A0843120E10431B4A9062B4352B680F490B6068684860A8688860E868C86016490B68DB0608D4306A012189030843306202E00024124908600120400620430D49086006B0F0BD5C000F00608B0E00089A0E0020200000801100048031800480318044800D800420020100400031
:6E8ACA00020068D208000004000164830E0008800E00189A0E00104A1068102108400023002800D101230D4A1078184013D00C49086800230B6003235B040A490B600B60084908600023137004490B68DB0602D501230548C3777047C04608800E00619E090064830E005C000F002422080079
:FB8B4000F0B585B0061C75680495B0780207130F0093F2780292C02101408F11062B00D9A9E1CB4C2378CB490879834202D3201CAEF76EFDC7484188002923D00378002B10D06378002B04D0C34899F73DFB002818D000236370A370BE4A508850214143BD4805E02378BC48002B04D15022514399F7DFFA06E099F727FB002802D0201CAEF746FD20782923191C41430191E11C8807800F01D10A6808E0091AC0000B68C3402022101A4A6882401A4301988018AA49009A515C0170032A01D0052A51D1A74A13681B0600D438E14770029A931F0372291C09300622BCF706F90635291CE21C9007800F01D1136808E0121AC0001768C7402023181A5368831D
:FB8C3B00403B430198C318981C0622BCF7EFF80098052817D10635029A0C3A291CE31C9807800F01D11F6808E01B1AC0001D68C5402027381A5F6887402F430198C0190F30BCF7D4F8E11C8807800F01D10B6808E0091AC0000A68C2402023181A4B688340134301990F1CE1E0FF07FF0F0098042806D07D4A13687068F1784018C078587279490868C379012B1BD1391C281CAEF7F1FF009A042A05D1AFF70EF8002800D1CEE04DE0011CFF2904D1391C281CAFF736F8011C081CAFF714F8002800D1BFE03EE06A490B78002B3AD0009A042A16D167480390291C1030062200F045FF002800D0ADE00399887D03071B0FBB4200D0A6E0010600D4A3E0400650
:FB8D3600400E1EE00922835601200856834200DA99E058480390291C1030062200F027FF002806D10399887D03071B0FBB4200D189E0291C039810300622BCF75AF8802038430399887501210391E11C8807800F01D10A6808E0091AC0000B68C3402022101A4A6882401A43019880184770291C02300622BCF73DF839480378002B1CD0F07871684318191CE21C9007800F01D1136808E0121AC0001768C7402023181A536883403B430198C018AFF7D5F80006000EFF2801D0002103910098042808D12A490B681B0604D429490B685879002839D00398002836D00635029FFA373F063F0E0297E11C8807800F01D10B6808E0091AC0000A68C24020231834
:898E31001A4B6883401343019FF818029A0272291C0930BBF7F0FFE11C8807800F01D10B6808E0091AC0000A68C2402023181A4B6883401343019FF81828307368F1785B18DB780370237801332370237805490879834214D3201CAEF7E2FB10E0C04657C80800B4A208008DC80800B8E30500A82D08007851080062C808000CA30800049898F735FC05B0F0BD8B
:FB8EC000F0B587B0041C4E680C36371C032301A80370251CA8352878002815D0022858D9052800D299E000D1CAE0072800D2D3E000D1F8E00E2800D23EE100D1DCE0102818D300D1E8E037E1032A00D034E1201C8830B3F758FF201C9030B3F766FF236B8020034323639B0603D42021A87DB3F70FFCF7E0112A00D01EE10822211C943101A80130BBF770FF211CA43101A809300222BBF769FF0822211C883101A80B30BBF762FF211C903101A813300422BBF75BFF172201A9A87DB3F7BEFBD64803681B0703D5236B9B0600D5F2E001232B70F2E0042A5FD10822791C201C7C30BBF743FF391C0931201C84300422BBF73CFF0822211C8831201C5430BBA9
:FB8FBB00F735FF0822211C7C31201C5C30BBF72EFF211C9031201C74300422BBF727FF211C8431201C78300422BBF720FF221C6432211C5431201C4430B0F791FB211C6431201CAFF7D9FD211C7431201CAFF7E0FD04202B78012B00D0AFE00320ADE0052A1BD181B000200090019008BCA87D00210A1CB0F749FB236B102003432363A87D0321B0F7D2FA201CB3F7BAFA06202B78032B00D091E005208FE00D2A00D08DE0236B102083432363A87D0021B0F7BDFAA87DB2F77EFF7178201C0022AEF727FC002386E7062A79D1201C01220021AEF71EFCA87DB2F76DFF0E237AE7062A6DD1201C0021AEF72CFCA87DB2F762FF0E232B70236B80208343236394
:FB90B6005FE0032A5DD12021A87DB3F746FB201C8830B3F77DFE201C9030B3F78BFE102326E0112A4DD1201CB3F771FA072353E70B2A46D1236B102083432363A87D0021B0F776FA201CB3F766FA754A13681B0713D500F034FD061CA87D0121B2F721FF301C00F034FD236B2020034323630F232B70A87DB2F705FF23E00822211C943101A80130BBF775FE211CA43101A809300222BBF76EFE0822211C883101A80B30BBF767FE211C903101A813300422BBF760FE172201A9A87DB3F7C3FA02230BE7287007B0F0BD70B584B0041C4E680C36042368460370251CA8352878002816D0082800D29EE100D1BBE0092800D1C7E00C2800D2CFE000D104E10E5A
:FB91B1002800D221E100D1E6E010285ED300D1EFE08AE1032A00D087E1444A1178201CCB0703D41A21B3F73DFA7EE17C30B3F7F2FD201C8430B3F700FE0822711C201C9430BBF719FE311C0931201CA4300222BBF712FE0822311C0B31201C8830BBF70BFE311C1331201C90300422BBF704FE0822211C8831201C5430BBF7FDFD0822211C7C31201C5C30BBF7F6FD211C9031201C74300422BBF7EFFD211C8431201C78300422BBF7E8FD211C7431201CAFF7B5FC236BFF200130034323635B0603D42021A87DB3F76CFA0F238DE0112A00D02BE10822211C7C3168460130BBF7CCFD211C8431684609300422BBF7C5FD0D226946A87DB3F728FA0D48806A89
:FB92AC0000220121490701400A4303D00A4A5268D0061ED4236B5B06DB0F201C002B0ED00622111CB3F786F808E0C0465C14080008960800D8200800A048080001E0B3F7BDFD00232B70236BFF20013083432363EDE0201CAEF7BBFA7C490B681B0703D5236B5B0600D5E0E00823DFE00E2A04D1201CB3F77EFD0A23D8E00F2A00D0D6E0201CB3F79BFD0023D0E00E2A04D1201CB3F76FFD0B23C9E00F2A00D0C7E0BBE0062A00D0C3E0236B102003432363A87D0321B0F742F9201CB3F72AF9A87DB2F700FE2B78201C00210A2B03D10122AEF7A6FA01E0AEF7BCFA0E23B3E70A2A00D0A5E02021A87DB3F7DDF910232B70A87DB2F7CCFD9BE0112A00D098BA
:FB93A700E0A87D0121B0F71BF9201CB3F70BF90C238EE00B2A00D08CE0236B102083432363A87D0021B0F70BF9494A13681B070ED500F0CCFB061CA87D0121B2F7B9FD301C00F0CCFB236B4020034323639DE70D236EE0032A6DD1201C7C30B3F7E0FC201C8430B3F7EEFC0822711C201C9430BBF707FD211CA431301C09300222BBF700FD0822311C0B31201C8830BBF7F9FC311C1331201C90300422BBF7F2FC0822211C8831201C5430BBF7EBFC0822211C7C31201C5C30BBF7E4FC211C9031201C74300422BBF7DDFC211C8431201C78300422BBF7D6FC211C7431201CAFF7A3FB0822211C7C3168460130BBF7CAFC211C8431684609300422BBF7C3FC9D
:6294A2000D226946A87DB3F726F91348806A00220121490701400A4303D0104A5268D00605D4201C0622111CB2F789FF30E7201CAEF7D2F909232B7004B070BD00B5002808D0BD231B5C002B02D1FFF7E8FC01E0FFF743FE00BD5C140800D8200800A048080051
:7095080000B5417C18224A43174951180A23CA56002A03DD013A8A72B2F759FC00BDF0B5061C20D03768002F1DD0707CADF75CF8051C707C182141430B484418786890F740FA98F72FF9381C98F7E6F800233360217A01312172217A04480278A88D90F775F900232372F0BDA8B5080098140800A1
:FB95840070B581B0061C00236A46D370341C0834C81C74F7E9F8051C05D0EB691B06DB0ED81F052802D3122333700DE069460331286873F770FE6A46D378E371FF200530285CA0710223F37001B070BD00B5CB78B04803700431B0480622BBF723FC00BD30B5051C0B79AD4A1370CB78AC4A1370AC4C201C74F7B8F8A94A1378002B16D0A9498B79022B02D10D232B7011E000280FD1A648017F00290BD1A54B1970A54B1A88A54B1968201C85F7CAFE01E07BF71DFC30BDF0B586B0A04CA1490B689B0500D4D4E0002103919E4DEB691806C00EDB0200D4C0E0F8214B595B0700D5BBE0072802D0092800D0B6E0002104910591039801300190012686408681
:FB967F00480378002B08D08549281C2830062200F089FA002800D1A1E0281C74F7EFFD002820D069460331019873F7DAFD281CF023C156F0306B4603229A56844B02938B1A082701B40398C75701BCBB4209DB029F7B785B421B061B16994202DA012304930593027001990F191237B87B002803D00138B87300061AD1744A0292D078002803D1608A304012D00FE001280FD169460231019873F7A4FD029A0020135658426A4602215356834201DA01210491208A304005D0B878002808D00138B87005E062490B79BB70208A30432082BB78002B10D1A08D30400DD05C498B78BB73608AB0436082608921890840A1890840304020D033E00498002830D0E4
:FB977A00608821880840A1880840304029D1059A1F21281C7BF720F8002822D0281C74F770FD00281DD12089B04320814A4BE95C002916D00139E95413E02021281C00227BF70AF800280CD0281C74F75AFD002807D12388B34323803F4BE818037801330370FF230933ED180398013003900B2800D22FE70020A08506B0F0BD70B583B005250622354901A8BBF711FB284E01A9301C062200F0C9F9002800D185E0301C73F7A7FF041C13D02D480378002B7CD101230370E3691B06DB0ED81F05281AD269460331206873F72BFD2248205C1AE01948037F002B0ED114480378002B64D01748028817480168301C85F7AEFD00231248037059E010490023C895
:FB98750056002854D06946C87000206A4603215156154B1A5691423DDA7F23DB43994224E0C046C1C50800629E0900C9C50800C8C50800C2C5080038460800B8210800ED070800F4070800F00708000ECA08009C1B0800883608001C04080004010000D29B09007E9C0900CAC5080013DD4D490878013008700878E3691B06DB0E092B00D10325A84213D347480378002B0FD092F7EEF90CE0454B1856814205DD44480378002B01D092F7C8F900233D48037003B070BC08BC1847F0B581B0051C00913C4E7BF7AEF8A02148552C1C6434227F111C371CF8373B79002B0DD07B798B420AD1BB79F854BB79581C43109B0F1B189B109B00C01AB871101C74F7B6
:CC99700028FA002808D02D492830062200F012F9002801D12A4908702F1C217F9F2038569F377BF754F83870271CBB7D0C37002B14D02368DB0507D433691B010ED5201C90F771FB002809D00023A3610123FB720023BB727B72201C8EF7C5FB23685806000F00990A5C002A05D0164B185CA072431EAB8115E03369DB000BD512490A6811684B031B0F984204D18B025B0F581EA88106E0012323723B68FF20013083433B6001B0F0BDC0467D9C0900C9C50800DEC50800C8C50800D8200800C2C508007E9C090072BF0500E02908006A
:E49A4C0030490B68082003430B600B6883430B60704770B500242C4E3378002B07D12B4D286B002801D097F79BFE2C636C632848847628480378002B0CD0202326490B60A3F77AFA25490B78002B01D1A3F7BCFA204804708CF79FFF002802D03378012B01D1A1F79EFF70BD01231D480370704700B518480378002B01D0FFF7C1FF002317490B7008208DF724F800BD00B514480378002B05D120230F490B60A3F74CFA02E001230B48037000BD0D480378002B03D10748837E012B01D1002000E001207047C04608330E00586A08003C6808005C680800809C090014000C0032C808007F9C0900F0
:FB9B74007847000000C09FE51CFF2FE178D504007847000000C09FE51CFF2FE18CD504007847000000C09FE51CFF2FE1704D05007847000000C09FE51CFF2FE13C4B050091000000F797090092000000000000000000000000000000000000000000000000000000140F14061A001FAD00000000C0A9000027AA000004AA000009AA00000EAA000013AA000018AA00001CAA000022AA00009855000040550000B155000084550000895500008E550000935500009D550000A2550000A7550000AC550000B65500003B5500000F21032328410E42430000001C000000597A0900EF7C0900D3AE040000000000237D090000000000977B0900B77D09005FB10416
:0B9C6F0000ADB1040011AF04006C0256
:029C7F000000E3
:00000001FF
